:100000000C9498010C94D0010C94D0010C94D00164
:100010000C94D0010C94D0010C94D0010C94D0011C
:100020000C94D0010C94D0010C94B31B0C94851C3F
:100030000C94A7160C94D0010C94D0010C94D00110
:100040000C94D0010C94D0010C94D0010C94D001EC
:100050000C94D0010C942F170C94D0010C94D00167
:100060000C94D0010C94D0010C94D0010C94D001CC
:100070000C94D0010C94D0010C94D0010C94D001BC
:100080000C94D0010C94D0010C94D0010C94D001AC
:100090000C94D0010C94D0010C94D0010C94D0019C
:1000A0000C94D0010C94D0010C94D001530453044F
:1000B00086048604AD04D704D705D705E9047E0578
:1000C00090059005F21C191D111E191D111E651DAC
:1000D000881D111EDF1DEE1D29001E001F002000BF
:1000E00021002200230024002500260027002D00E7
:1000F0002E0000002A002B0014001A000800150032
:1001000017001C0018000C00120013002F00300014
:1001100031000000390004001600070009000A0041
:100120000B000D000E000F0033003400000028000B
:100130000000E10000001D001B0006001900050082
:10014000110010003600370038000000E500000004
:10015000E000E300E2000000000000002C000000CE
:1001600000000000E60001516500E40000003500D9
:100170003A003B003C003D003E003F004000410093
:10018000420043004400450000000100010001005E
:100190005200010001000100010001004B004E006F
:1001A00046004700480001000000010050005100D7
:1001B0004F000100010001000100010001000100E9
:1001C000010000000100000001000000010001002A
:1001D0000100010001000100010001000100010017
:1001E000000001000000010001000100000000000B
:1001F00000000100000000000000010001000100FB
:10020000010000000C035300360030002D005800A0
:1002100000001003530065006E007400720061005E
:10022000710000000403090409023B00020100A060
:10023000FA09040000010301010009211101000174
:1002400022400007058103080001090401000103A1
:10025000000000092111010001227B000705820333
:100260002000011201000200000008EDFE606001A4
:10027000000102000105010902A10185020901A195
:100280000005091901290815002501950875018146
:10029000020501093009311581257F950275088114
:1002A0000609381581257F950175088106050C0A18
:1002B00038021581257F950175088106C0C00501AA
:1002C0000980A101850319012AB700150126B7008D
:1002D000950175108100C0050C0901A10185041963
:1002E000012AA002150126A002950175108100C007
:1002F00005010906A101050719E029E715002501F7
:10030000950875018102950175088101050719009D
:1003100029FF150026FF00950675088100050819BC
:10032000012905950575019102950175039101C09B
:1003300011241FBECFEFDAE0DEBFCDBF04B603FE4F
:1003400018C080917B0290917C02A0917D02B091B7
:100350007E028730904BA740B04B59F410927B023D
:1003600010927C0210927D0210927E02E0E0F8E38F
:10037000099511E0A0E0B1E0E8E8FDE302C00590D6
:100380000D92A039B107D9F722E0A0E9B1E001C090
:100390001D92AB37B207E1F70E94FC100C94C21E0D
:1003A0000C94000081E0089581E008950C94D4013C
:1003B00008950C94D8011F93CF93DF9300D000D001
:1003C0001F92CDB7DEB749835A836B833091930177
:1003D00089819A81311114C0662359F0222349F092
:1003E0000E94F107182F682F89819A810E949A072D
:1003F00003C00E94C507182F69817A81812F04C02C
:100400000E94F10769817A810F900F900F900F90F1
:100410000F90DF91CF911F910C94670EFC01262F56
:10042000408151816281738184810C94DB0181E080
:100430000895CF93DF93EC0160E00E940E02BE01AD
:10044000DF91CF910C94D9010C94AD0F0C94A90FAE
:1004500008950E9444060E9428022FEF84E39CE046
:10046000215080409040E1F700C000000C945517E7
:100470000F931F93CF93DF93EC0161E00E940E0274
:100480008C01BE010E94D601882349F1BE01C8013A
:100490000E947E15882319F1BE01C8010E949213A3
:1004A0008823E9F0BE01C8010E94DA148823B9F05C
:1004B0008A81882369F001158CE5180731F00F3D1A
:1004C0001C4531F40E94860C0AC00E94290207C014
:1004D000CE01DF91CF911F910F910C94D20180E05A
:1004E000DF91CF911F910F9108950E9489160C946E
:1004F0008E020E9491020C948F1608950C947D0236
:1005000081E008950C9480020895CF93C82F0E9433
:100510007E028C2F0E948202CF91089580E00C947D
:1005200085020E94DA150C9485020E94DA159091DA
:100530009201891721F0809392010C94850208950D
:10054000CF93DF93CDB7DEB72B970FB6F894DEBF0E
:100550000FBECDBF4F83588769877A878B8761111C
:100560000E94D50B9E012F5F3F4F86E0F90111924B
:100570008A95E9F785E0FE013796D90101900D9241
:100580008A95E1F789819A814C815D81452B31F013
:100590009F3F31F491E08F3F19F403C091E001C017
:1005A00090E090FF09C049815A816B817C818D81E7
:1005B0009E810E94D80A05C0C9010E9417028111BC
:1005C000F2CF2B960FB6F894DEBF0FBECDBFDF91F2
:1005D000CF910895FC01808191810E943308089594
:1005E000CF93882309F4A4C0C82F8238C1F40E9495
:1005F000DA1581FD9DC069E38091020190910301AC
:100600000E9461160E94860B2FEF81EE94E021502C
:1006100080409040E1F700C0000069E319C08338D2
:1006200001F50E94DA1580FD83C063E58091020127
:10063000909103010E9461160E94860B2FEF81EEBC
:1006400094E0215080409040E1F700C0000063E555
:1006500080910201909103010E946316CF910C9446
:10066000860B8438C1F40E94DA1582FD61C067E40C
:1006700080910201909103010E9461160E94860BF5
:100680002FEF81EE94E0215080409040E1F700C0D0
:10069000000067E4DDCF8CEF8C0F813AD0F46C2F33
:1006A00080910201909103010E942B16882349F04A
:1006B0006C2F80910201909103010E9463160E94A9
:1006C000860B6C2F80910201909103010E946116AC
:1006D000C5CF80E28C0F883048F4C77081E001C03C
:1006E000880FCA95EAF70E94B80BB8CFEBE5EC0F7C
:1006F000E33040F4F0E0E95BFE4F808190E0CF9181
:100700000C94FF15E8E5EC0FE73150F4F0E0EE0F44
:10071000FF1FE75EFE4F80819181CF910C941516EB
:10072000CD3E30F08C2F0E948111CF910C9453124A
:10073000CF910895882309F464C0823879F40E9427
:10074000DA1581FF5EC069E3809102019091030197
:100750000E9461160E94860B69E310C08338B1F4D1
:100760000E94DA1580FF4DC063E5809102019091EF
:1007700003010E9461160E94860B63E580910201CD
:10078000909103010E9463160C94860B843879F4CF
:100790000E94DA1582FF35C067E4809102019091D2
:1007A00003010E9461160E94860B67E4E7CF9CEF6D
:1007B000980F913A10F4682FE1CF90E2980F98309B
:1007C00050F4877091E001C0990F8A95EAF7892F5C
:1007D0000E94BE0BD9CF9BE5980F933020F480E0A8
:1007E00090E00C94FF1598E5980F973120F480E085
:1007F00090E00C9415168D3E20F00E94DC110C94B4
:10080000531208951F93CF93DF93182FEB010E948B
:10081000F002209741F08FE99FE00197F1F700C0C7
:1008200000002197F6CF812FDF91CF911F910C947B
:100830009A03893319F060E070E002C060E570E06F
:100840000C940204882321F00E94B80B0C94860BB0
:100850000895882321F00E94BE0B0C94860B089506
:10086000CF92DF92EF92FF920F931F93CF93DF937C
:10087000DC01C62F972F12962C91129715964C914A
:100880001597342F32953F70172F12951F70C12E78
:10089000D12C8CE0C816D10408F089C1F601EA5ABF
:1008A000FF4F0C94591E872F807F9F70D92F88236C
:1008B00011F0D295D07F222399F0DD2309F463C192
:1008C00080E28C0F883010F0C11104C08D2F0E947F
:1008D000B80B03C08D2F0E94C80B0E94860B53C11A
:1008E0008C2F0E949A03DD2309F461C180E28C0FF2
:1008F000883010F0C11104C08D2F0E94BE0B03C0C0
:100900008D2F0E94CE0B0E94860B51C1872F807FB6
:100910009F70803211F4892F03C0892F8295807FC8
:10092000C13051F4222321F0363008F040C10DC00F
:10093000353008F03CC10EC0222351F0332329F09A
:1009400040FF21C14F7015964C930E9422042FC185
:1009500031111FC10E9429042AC1872F86958695CF
:10096000837019F0813091F022C1222319F0862F73
:10097000937002C080E090E0DF91CF911F910F91C2
:10098000FF90EF90DF90CF900C94FF15222319F089
:10099000862F937002C080E090E0DF91CF911F918D
:1009A0000F91FF90EF90DF90CF900C941516862F4B
:1009B000222319F00E94811102C00E94DC11DF91F4
:1009C000CF911F910F91FF90EF90DF90CF900C94FB
:1009D0005312872F837009F045C02111EBC0862F79
:1009E000829586958770880F880F462F4F7050E04C
:1009F00060E070E0082E04C0440F551F661F771F8B
:100A00000A94D2F7C4FF10C00FE010E020E030E0FD
:100A100004C0000F111F221F331F8A95D2F70095C3
:100A200010952095309503C000E010E09801969550
:100A30009695E92FE370CB01BA01602B712B822BC5
:100A4000932BE23049F058F4E13019F00E94B006DF
:100A5000B1C00E949E06AEC00E94C206ABC00E94FA
:100A60009C06A8C0222319F0872F817001C08695AB
:100A7000882309F49FC08C2F829586958770880FF4
:100A8000880F4C2F4F7050E060E070E0082E04C0DB
:100A9000440F551F661F771F0A94D2F7C4FF10C07A
:100AA0000FE010E020E030E004C0000F111F221F13
:100AB000331F8A95D2F7009510952095309503C085
:100AC00000E010E0980196959695E92FE370CB0130
:100AD000BA01602B712B822B932BE23049F058F432
:100AE000E13019F00E94750765C00E94630762C07B
:100AF0000E9487075FC00E94D6065CC0D72FDF70B8
:100B0000222339F08D2F0E94FC068C2F0E94220494
:100B100051C0862F0E9429048D2F0E941D074AC0B4
:100B2000613FA9F018F4603F31F029C0623FB1F095
:100B3000633FD9F024C0222339F03530C0F5892F26
:100B40008F710E94420733C0363088F5F8CF2223D8
:100B500039F0892F8F710E94FC0629C02223C9F326
:100B6000892F8F710E941D0722C0222329F0872F11
:100B70008F710E94E7061BC00E94E20618C0222364
:100B800031F0332331F38C2F0E94F00210C0332355
:100B900039F3C93349F49FEF27EE83E091502040A9
:100BA0008040E1F700C000008C2F0E949A0318508B
:100BB000143060F40E94DA15DF91CF911F910F91EC
:100BC000FF90EF90DF90CF900C948502DF91CF9152
:100BD0001F910F91FF90EF90DF90CF9008950F93AA
:100BE0001F93CF93DF93EC01688179818A810E9402
:100BF0003E088C010E9499070E948A06B801CE0126
:100C00000E943004DF91CF911F910F910895CF93EF
:100C1000DF93FC019081818123813481232B31F08A
:100C20008F3F31F481E09F3F19F403C081E001C0A0
:100C300080E080FD0EC0EF01CF010E9438028823C2
:100C400041F0CE010E94EF05CE01DF91CF910C94CF
:100C50001902DF91CF91089580E090E00E94FF1586
:100C600080E090E00E9415160E94D50B0E94860B32
:100C70000E9484130C9453128091020190910301FD
:100C80000E9465160C942C060E94C50B0C943C0621
:100C900092959F70963079F010F4925001C09A505E
:100CA000923068F4803F69F018F4883E40F409C03F
:100CB000843F29F406C0883E20F0813F11F080E097
:100CC000089581E00895FC01808191810E9433089C
:100CD0000E9448060895CF93DF9300D000D01F9262
:100CE000CDB7DEB70F900F900F900F900F90DF9160
:100CF000CF910895CF93DF9300D000D000D0CDB72F
:100D0000DEB726960FB6F894DEBF0FBECDBFDF91DB
:100D1000CF910895089508950C948B060C948C0639
:100D20000E948E066093CA017093CB018093CC0120
:100D30009093CD010C942C060C9490060F931F9366
:100D40000091CA011091CB012091CC013091CD01CD
:100D5000602B712B822B932B1F910F910C9490067B
:100D60000F931F930091CA011091CB012091CC01E8
:100D70003091CD0160237123822393231F910F9122
:100D80000C9490060F931F930091CA011091CB0110
:100D90002091CC013091CD016027712782279327C4
:100DA0001F910F910C9490060C948B060E94D40610
:100DB0006093C6017093C7018093C8019093C901E5
:100DC0000C942C0660E070E0CB010C94D6060F93D7
:100DD0001F9341E050E060E070E08A019B0104C095
:100DE000000F111F221F331F8A95D2F7C901B801C6
:100DF0001F910F910C94D6060F931F9341E050E082
:100E000060E070E004C0440F551F661F771F8A958D
:100E1000D2F78091C6019091C701A091C801B0910D
:100E2000C9018A019B01082B192B2A2B3B2BC901D5
:100E3000B8011F910F910C94D6060F931F9341E0B8
:100E400050E060E070E004C0440F551F661F771F3C
:100E50008A95D2F740955095609570958091C6011E
:100E60009091C701A091C801B091C9018A019B016D
:100E7000082319232A233B23C901B8011F910F918D
:100E80000C94D6060F931F9341E050E060E070E0B1
:100E900004C0440F551F661F771F8A95D2F78091B3
:100EA000C6019091C701A091C801B091C9018A0102
:100EB0009B01082719272A273B27C901B8011F9141
:100EC0000F910C94D6060F931F930091C6011091B9
:100ED000C7012091C8013091C901602B712B822B71
:100EE000932B1F910F910C94D6060F931F93009193
:100EF000C6011091C7012091C8013091C90160233A
:100F00007123822393231F910F910C94D6060F9384
:100F10001F930091C6011091C7012091C801309123
:100F2000C90160277127822793271F910F910C9485
:100F3000D60608952FE0929F800D1124E82FE695A4
:100F4000E695E695877051E001C0550F8A95EAF75E
:100F500085E0E89FF0011124EC56FE4F20E030E0E0
:100F600070E04081CB01022E02C0969587950A94CD
:100F7000E2F78170819584278523842781932F5FF1
:100F80003F4F2530310569F708952FE0929F800D7E
:100F90001124682F669566956695982F977085E061
:100FA000689FB001112440E050E080E0FB01E40FB5
:100FB000F51FEC56FE4F208130E0092E02C0369519
:100FC00027950A94E2F721703327042E01C0220FDF
:100FD0000A94EAF7822B4F5F5F4F4530510531F796
:100FE0000895BF92CF92DF92EF92FF920F931F93DB
:100FF000CF93DF938C01C090C601D090C701E090E1
:10100000C801F090C9018091CA019091CB01A091D3
:10101000CC01B091CD01C82AD92AEA2AFB2ACFE116
:10102000D0E0D701C6010C2E04C0B695A7959795C0
:1010300087950A94D2F780FD04C0219790F7B12CD0
:1010400007C0BC2EB8018C2F0E947A0E0197A9F31D
:101050008B2DDF91CF911F910F91FF90EF90DF903B
:10106000CF90BF900895CF93DF93EC010E94F107DA
:10107000BE010E947A0EDF91CF9108951F93CF9306
:10108000DF93EB0190919301992321F0CB010E9412
:10109000330813C0882349F0CB010E94F107182FB1
:1010A000682FCE010E949A0704C0CB010E94C50799
:1010B000182FBE01812F0E947A0EDF91CF911F91D0
:1010C00008951F93CF93DF93C091CE0116E08091D6
:1010D000CF01C81799F0D0E01C9FF0011D9FF00DC3
:1010E0001124E053FE4F40815181628173818481DC
:1010F00095810E947A062196C770E9CFDF91CF9142
:101100001F910895409100025091010260910202E6
:101110007091030280910402909105020C947A066A
:10112000EF92FF920F931F93CF93DF93809105026D
:1011300082958F7009F065C080910202882309F4BE
:1011400060C08091CE01F090CF011091000200911B
:101150000102609103027091040291E01F3F09F0C7
:1011600090E0C0910001D0910101292F96E0E92E75
:101170008F1509F446C06115710521F00F3F21F06C
:1011800030E003C031E001C0322F90E030FD36C0C6
:10119000E89EF001E99EF00D1124DF01A053BE4F3F
:1011A00011963C911197301329C03C91311326C000
:1011B00012963C911297311121C013964D915C917A
:1011C0001497461B570B4C175D07C0F4809105021E
:1011D0008F70806180930502EB52FE4F80818F708B
:1011E0008061808380E092E00E940706DF91CF91CA
:1011F0001F910F91FF90EF900C94610801968770FA
:10120000B7CFDF91CF911F910F91FF90EF9008958D
:101210009F92AF92BF92CF92DF92EF92FF920F9385
:101220001F93CF93DF93CDB7DEB761970FB6F894D6
:10123000DEBF0FBECDBF8C0185E0F801DE011D963B
:1012400001900D928A95E1F7D8011296EC90909159
:101250000002E09101022091030230910402211565
:10126000310531F0EF3F31F481E09F3F19F403C0C5
:1012700081E001C080E0B82FB1709B2E80FD47C196
:10128000D8014C9111965C9111971396AD90BC903A
:10129000149780E0C82E82E0D82EF0900202B501AB
:1012A000621B730B2091000130910101FF2009F4B2
:1012B000D9C0809105026217730708F095C0282FE6
:1012C000207F09F052C05E1313C0491311C0FE2CD9
:1012D000E1100EC08F708061809305020E94820829
:1012E000C6010E94070680910502F80185834DC161
:1012F000AB2831F05F3F31F481E04F3F19F403C078
:1013000081E001C080E080FD03C081E08E2502C045
:1013100080E090E0F82FF170FF2E80FF1CC08091DC
:10132000CE012091CF0136E0821709F40BC190E085
:10133000389FF001399FF00D1124E053FE4F618179
:10134000561306C06081461303C06281E61203C0D3
:1013500001968770E9CFFE2CEE2009F416C180912A
:10136000050281608093050254C05E1306C04913D4
:1013700004C0E11002C0F80199C0C8010E946306D0
:10138000882361F1EE2051F120910502822F829590
:101390008F7090E0029774F08091000290910102AA
:1013A00098878F831986BB86AA862C87CE010796DD
:1013B0000E94070686E0F801A0E0B2E001900D92DD
:1013C0008A95E1F70E9490080E9482080AC05E1781
:1013D00011F1C8010E94630681112CC0C8010E944E
:1013E0000706FF24F394D1C0282F207F81F77A2DA0
:1013F000B98AA88A6E2D89890E946B0680E092E0E6
:101400000E94070686E0D6011D928A95E9F70E94A0
:101410008208F12CBAC04913DCCFE110DACFF80111
:101420008583C8010E94070686E0D6011D928A9531
:10143000E9F7ABC0EE2091F220910502822F829550
:101440008F7090E002970CF4B5CF809100029091DC
:1014500001029A8389831B82BD82AC822E83CE01D6
:101460000196A6CF6217730708F044C0FE2CEE2049
:1014700009F4B4CF5E1330C049132EC02091050289
:1014800020FD21C0822F82958F70482F50E041159A
:101490005105C9F0F80125834F30510541F08F5FA8
:1014A000982F9295907F822F8F70892B8583C8010A
:1014B0000E94070686E0F801A0E0B2E001900D92DC
:1014C0008A95E1F73CC086E0F801A0E0B2E0019027
:1014D0000D928A95E1F759C0C8010E9463068111F7
:1014E00069CF80910502816080930502C8010E9446
:1014F00007064BC07A2DB98AA88A6E2D89890E9469
:101500006B0686E0D6011D928A95E9F718C0EE2099
:1015100009F464CFC8010E946306F82E882309F4F9
:101520005DCF86E0F801A0E0B2E001900D928A95CF
:10153000E1F780E092E00E94EA020E9490080E9497
:10154000820823C04D875E878D859E850E94330863
:10155000292F22952F70223028F49F7039F08111A5
:1015600005C00BC0243028F49F7049F4805E883099
:1015700020F0C8010E9407069F2CF92C06C0D80154
:1015800015969C91907F91F7F8CF8F2D61960FB6AD
:10159000F894DEBF0FBECDBFDF91CF911F910F91A9
:1015A000FF90EF90DF90CF90BF90AF909F90089505
:1015B0001F93CF93DF93CDB7DEB72C970FB6F89478
:1015C000DEBF0FBECDBF4F83588769877A878B8771
:1015D0009C87CE0107960E9408098823D1F09F813D
:1015E00088852A853B85232B31F08F3F31F481E0BC
:1015F0009F3F19F403C081E001C080E080FD47C037
:101600004F81588569857A858B859C850E947A06ED
:101610003EC086E0FE013796DE01119601900D92E4
:101620008A95E1F7FF81E8856A857B8561157105FB
:1016300031F0EF3F31F481E0FF3F19F403C081E066
:1016400001C080E080FD23C02091CF0130E0C901BE
:101650000196877099274091CE0150E08417950735
:10166000F1F1F983EA837D836C8396E0929FD00148
:10167000939FB00D1124A053BE4FFE0131960190EF
:101680000D929A95E1F78093CF010E94610816E0D0
:101690008091CE019091CF01891771F1189FC001FF
:1016A000112480539E4F0E940809882329F1E0915C
:1016B000CE011E9FF0011124E053FE4F4081518165
:1016C00062817381848195810E947A068091CE0126
:1016D00090E00196877099278093CE01D9CF0E9420
:1016E00044061092CF011092CE01E0E0F2E086E0D5
:1016F000DF011D928A95E9F72C960FB6F894DEBFAC
:101700000FBECDBFDF91CF911F910895CF93DF938F
:10171000E0910201F0910301809117028083E09132
:101720000201F0910301908180911602892B808340
:10173000C0910201D091030148E050E066E072E000
:10174000CE010E94731E892B69F088E0FE01A6E09D
:10175000B2E001900D928A95E1F7CE01DF91CF9131
:101760000C94E615DF91CF910895809117020895AA
:1017700090911702892B809317020895809590917C
:101780001702892380931702089510921702089573
:1017900090911602892B809316020895809590915E
:1017A0001602892380931602089510921602089556
:1017B0006FEF7FEF80E090E00C94AC1E80E090E053
:1017C0000E94881E21E0893E9E4F09F020E0822F72
:1017D000089582E090E00C94801E83E090E00C94E9
:1017E000801ECF9384E090E00E94801EC82F82E28A
:1017F00090E00E94801E2C2F30E0A901582BCA01D6
:10180000CF910895CF93C92F682F84E090E00E9474
:101810008E1E6C2F82E290E0CF910C948E1EAB0155
:10182000BC018FE090E00C94A01EAB01BC0183E1F1
:1018300090E00C94A01E60E070E0CB010C94150CBD
:1018400060E070E0CB010E940F0C0C941B0C69EE61
:101850007EEF80E090E00E94AC1E60E082E090E0CD
:101860000E948E1E60E083E090E00E948E1E109227
:10187000CA011092CB011092CC011092CD0160E010
:1018800084E090E00E948E1E60E082E290E00E9480
:101890008E1E60E085E090E00E948E1E60E086E093
:1018A00090E00E948E1E6FEF87E090E00E948E1EF7
:1018B00040E050E0BA0188E090E00E94A01E60E0A5
:1018C0008DE090E00E948E1E40E050E0BA0188E179
:1018D00090E00E94A01E60E087E190E00E948E1ED2
:1018E00040E050E0BA018CE190E00E94A01E60E070
:1018F00070E080E290E00E94AC1E40E050E0BA014F
:1019000088E190E00E94A01E0C94200C0C94270CFF
:10191000682F8EE090E00C948E1E0E941417609346
:1019200026027093270280932802909329026093E5
:10193000220270932302809324029093250208953B
:1019400085B7806885BF85B7806885BF089581E0C9
:1019500008950C94A70C08950C94AB0C0C94AB0C4C
:101960000C94AE0C0C94AB0C0C94B20C0C94AB0C11
:101970000E94A00C86E59FE00E94D0150E94B60C44
:101980000C94B40C0E94AC0C0C94AB0C0E94700F25
:101990000C9484020E94FF160E9455100E94C60CEF
:1019A0000C94B00C5F926F927F928F929F92AF9245
:1019B000BF92CF92DF92EF92FF920F931F93CF933C
:1019C000DF93CDB7DEB72A970FB6F894DEBF0FBE10
:1019D000CDBF0E946A10C82E81110E948D0C38E183
:1019E000832E32E0932E00E010E0502E802F0E94D4
:1019F000940F5C01F401619071904F016826792683
:101A000061147104B1F40F5F1F4F0530110569F7C0
:101A10008FEF89838A831B820E9408178160782F49
:101A20009D838C8349815A816B818D810E94A002A4
:101A30003AC080912A0281FD0E949D0FD12CEE2494
:101A4000E394F12CC3018E219F21892B29F10E945F
:101A5000A90C8823A9F0DE825F82AE20BF2081E03E
:101A6000AB2809F480E088870E9408178160782FEE
:101A70009A8789874E815F8168858A850E94A00246
:101A8000000F111FF801E85EFD4F80819181E8266B
:101A9000F926F182E08207C0D394EE0CFF1CFFE030
:101AA000DF12D0CFB0CF81E0C11001C080E02A9614
:101AB0000FB6F894DEBF0FBECDBFDF91CF911F915F
:101AC0000F91FF90EF90DF90CF90BF90AF909F90DD
:101AD0008F907F906F905F9008950E94D20C0E942B
:101AE00071120C949502CF93DF930E947F0EEC014C
:101AF000811520E5920768F5811530E4930708F019
:101B000098C08F3B910590F4883A910508F083C006
:101B1000853A910508F075C08430910508F0D3C06E
:101B2000019709F0CDC081E090E0CEC08F3F9105D4
:101B300009F050F48D3E910508F079C0805E91095E
:101B4000089708F4C0C0BCC08115904208F4BBC01F
:101B5000B7C0811554E5950780F5C11583E5D80711
:101B600008F087C0C11522E5D20708F06CC0C11586
:101B700031E5D30708F061C0CE0154E09695879512
:101B80005A95E1F7282F23703C2F337081E090E0C5
:101B900002C0880F991F3A95E2F79C68AC01522B5E
:101BA0009A019C2F9F709695969550E2959FE00123
:101BB0001124C9018C2B9D2B87C081154AE5940700
:101BC00080F4811559E5950708F069C0C11588E5CD
:101BD000D80708F475C0DC2FCC27CE01806F906A3F
:101BE00073C090568115904208F06AC08D2F8F7196
:101BF0000E94130FDD27D0628F71AE01582BCA01EE
:101C000063C0C55AD0E0C858DE4F8881C82FD0E0E5
:101C1000CE01906459C0C85AD0E0CC0FDD1FC65B1E
:101C2000DE4F0990D881C02DCE0194644DC09065DF
:101C30004BC0DF70CE01906A47C0DC2FCC27CE01AD
:101C4000816F906A41C0CE018370992721E030E016
:101C500002C0220F331F8A95E2F79C2F9695969526
:101C600080E2989FE0011124C22BD32BCE019C6807
:101C70002BC0CE018370992721E030E002C0220FF3
:101C8000331F8A95E2F79C2F9695969540E2949F94
:101C9000E0011124C22BD32BCE019A6815C08F709E
:101CA0000E94130F94E0D695C7959A95E1F7CF70EF
:101CB000D0E0DC2FCC27D0699E01282BC90104C0BD
:101CC00080E090E001C0CE01DF91CF9108952BE438
:101CD000829FC0011124FC012FE0729FE00DF11DD5
:101CE0001124E60FF11DEE0FFF1FE852FF4F859103
:101CF000949108950E94670E0E94730D0895823892
:101D0000910569F1B0F48133910509F46DC048F48F
:101D10008932910509F463C08A32910509F469C0DA
:101D200008958533910509F455C089339105B9F0BB
:101D30000895833E910569F138F4803E9105B1F034
:101D4000823E910509F10895863E9105A9F1873EED
:101D50009105B9F1843E910509F064C023C020913A
:101D6000540220FD4FC021FD4DC0089580915402C2
:101D700080FD44C08091550280FF44C08091540290
:101D800084FD42C083EE4DC08091540282FF38C072
:101D9000F5CF8091540282FD33C08091550280FDC1
:101DA00031C0ECCF8091550281FF32C08091540246
:101DB00084FD2AC087EE35C08091540283FF26C07F
:101DC000F5CF8091540283FD21C08091550281FDA1
:101DD0001FC0ECCF8091540285FD1CC01DC08091B6
:101DE000540285FD19C016C08091540286FD16C0AC
:101DF00017C08091540286FD13C010C089E311C042
:101E000082EE0FC080EE0DC080E00BC086EE09C0F0
:101E100084EE07C089E205C085E303C08AE201C001
:101E200081E390E008959091540292FF0DC0282F15
:101E30002871283019F4877F846006C0282F247108
:101E4000243011F48B7F886093FF0DC0282F2871F8
:101E5000283119F4877E846106C0282F247124312B
:101E600011F48B7E88612091550220FF0DC0382F20
:101E70003871383019F4877F816006C0382F31718E
:101E8000313011F48E7F886021FF0DC0282F28711A
:101E9000283119F4877E816106C0282F21712131F4
:101EA00011F48E7E886194FD877E089580E0089508
:101EB0000C94D80B0E946A108FE39CE90197F1F70C
:101EC00000C000000E946A1080E00E94940F80FF12
:101ED00004C00E94580F0C94551708950C945A0F83
:101EE0000E94DE0B811102C00E94860C0E94E90B49
:101EF00080932A020E94F10B909355028093540222
:101F00000E946E0F0E94ED0B682F70E080E090E061
:101F10000E949C066091C6017091C7018091C80122
:101F20009091C9010C94D406E82FF0E0EE0FFF1F4A
:101F3000E05AFD4F808191810895089580EA8A9545
:101F4000F1F7089500C008950C949E0F08950C9425
:101F5000A60F0C94A70F0C94A60F0C94AB0FF8943B
:101F6000E82FE295EF70F0E031A1282F2F7081E08B
:101F700090E001C0880F2A95EAF7982F9095932357
:101F800091A392A1892B82A3789408950F931F9314
:101F9000CF93DF93CAE8D1E089918F3F11F00E947F
:101FA000AF0F81E0CF38D807B9F7CBE7D1E00AE827
:101FB00011E089918F3F11F00E94AF0F0C171D07A0
:101FC000C1F7DF91CF911F910F910895BF92CF92EA
:101FD000DF92EF92FF920F931F93CF93DF938C01C9
:101FE000C62FD0E0CE0186579E4F6C01FC01908138
:101FF0009F3F09F450C0B62EF894E92FE295EF7098
:10200000F0E081A19F7021E030E001C0220F9A959D
:10201000EAF7822B81A382A12095282322A378941A
:102020000E94A20FEBE7F1E04AE851E021E030E046
:10203000E12CF12C61916F3F89F0A62FA295AF7032
:10204000B0E090968C9190E06F7002C09595879566
:102050006A95E2F780FD02C0C90102C080E090E00D
:10206000E82AF92A220F331F4E175F0719F7F601E6
:1020700080818F3F11F00E94AF0F61E0E114F10405
:1020800009F460E08B2D0E94A40FCC0FDD1FC00F60
:10209000D11FF982E882DF91CF911F910F91FF90BC
:1020A000EF90DF90CF90BF9008950E94C60F8AE016
:1020B000E0E6F2E0DF01982F1D929A95E9F7E6E558
:1020C000F2E0DF011D928A95E9F785E00E94B510E4
:1020D0000C942402FF920F931F93CF93DF93CDB7FD
:1020E000DEB72A970FB6F894DEBF0FBECDBF8E01C4
:1020F0000F5F1F4F8AE0F80111928A95E9F7F12CE2
:102100006F2DC8010E94E60FF394F5E0FF12F8CF9F
:102110004AE050E0B80186E592E00E94731EFF2479
:10212000F394009709F4F12C892B41F08AE0F8012F
:10213000A6E5B2E001900D928A95E1F72F2D45E0DA
:1021400060E672E086E592E00E94B6100E942602E8
:102150008F2D2A960FB6F894DEBF0FBECDBFDF914C
:10216000CF911F910F91FF9008950895FF920F93C3
:102170001F93CF93DF93F82E092F162FD72FC42F3D
:10218000222349F081E080932D020E94081790934A
:102190002C0280932B0280912D028823D9F080910C
:1021A0002B0290912C020E942017059798F0EF2D9A
:1021B000F02FA12FBD2F80E090E04C2F50E084172E
:1021C000950734F4219131912D933D930196F7CFEA
:1021D00010922D02DF91CF911F910F91FF900895E2
:1021E0000E940B190E94CA0C0C9417190E941B190B
:1021F0000E946D0D0C9435190E94A6160E94F218CB
:102200000E94B80C0E94F0100E94F6100E94C20CAE
:10221000FBCF8091340280FF06C06091090170E01D
:10222000660F771F26C081FF04C06091090184E01A
:1022300005C082FF07C06091090188E0689FB00176
:10224000112417C0909133029923D1F060910801B5
:10225000961788F72091090188E0289F90011124A2
:10226000929FA001939F500D112470E0CA010E941B
:10227000451E6038710540F46115710519F406C0FA
:1022800068E070E0862F08958FE7089581E0089553
:102290008091340280FF08C06091050170E075955F
:1022A00067957595679521C081FF06C0609105010E
:1022B00070E07595679519C082FF04C060910501B3
:1022C00070E010C090913202992399F0609104015E
:1022D0009617A0F780910501899FC001112470E035
:1022E0000E94451E6038710540F46115710519F4AE
:1022F00006C061E070E0862F08958FE7089581E0C1
:1023000008958D3E21F40E940911819504C08E3EEE
:1023100029F40E9409118093380208958F3E21F418
:102320000E940911819504C0803F29F40E9409117F
:10233000809337020895893F19F40E94481105C01F
:102340008A3F31F40E9448118195809339020895A3
:102350008B3F21F40E944811819504C08C3F29F4E1
:102360000E94481180933A0208959FE0980F983098
:1023700078F421E030E0A90102C0440F551F9A957E
:10238000E2F7CA0190913602892B809336020895B4
:102390008D3F21F48091340281600BC08E3F21F487
:1023A00080913402826005C08F3F29F4809134020D
:1023B00084608093340208958D3E39F49091380200
:1023C00097FF35C01092380259C08E3E29F4909183
:1023D00038021916BCF32BC0909137028F3E29F4B6
:1023E00097FF25C01092370249C0803F19F4191693
:1023F000CCF31DC090913902893F29F41916BCF421
:10240000109239023BC08A3F19F497FF10C0F8CFF1
:102410008B3F39F490913A0297FF09C010923A022B
:102420002DC08C3F21F490913A021916BCF39FE025
:10243000980F983080F421E030E0A90102C0440FE9
:10244000551F9A95E2F7CA0180959091360289232B
:102450008093360213C08D3F21F4809134028E7F29
:102460000BC08E3F21F4809134028D7F05C08F3FD9
:1024700029F4809134028B7F80933402809137025B
:10248000811106C080913802811102C0109233027E
:1024900080913902811106C080913A02811102C0F7
:1024A0001092320208950E940817209137022111DC
:1024B00004C020913802222321F0909331028093AE
:1024C000300220913902211104C020913A022223C6
:1024D00021F090932F0280932E0285E392E00C94DA
:1024E000F115EF92FF920F931F93CF93DF9300D0DC
:1024F00000D000D0CDB7DEB786E0E5E3F2E0DE0144
:10250000119601900D928A95E1F7E0903702F090D4
:1025100038020091390210913A021092370210925B
:1025200038021092390210923A02E11003C0FF20E3
:1025300009F45DC080913002909131020E94201711
:10254000AC0190913302992339F020910A0130E0D7
:102550002417350758F04BC020910B018AE0289FC3
:10256000900111242417350718F041C09F3F19F03E
:102570009F5F90933302EE2061F00E9409111E14B8
:1025800014F09FEF01C091E0989F902D112490933B
:102590003702FF2061F00E9409111F1414F09FEF11
:1025A00001C091E0989F902D1124909338023091B2
:1025B00037023323E1F0209138022223C1F045EBAA
:1025C0003403C0011124992319F09093370203C0FA
:1025D00081E08093370235EB2303C0011124992356
:1025E00019F09093380203C081E080933802011102
:1025F00003C0112309F45DC080912E0290912F0237
:102600000E942017AC0190913202992339F0209159
:10261000060130E02417350758F04BC02091070120
:102620008AE0289F900111242417350718F041C033
:102630009F3F19F09F5F90933202002361F00E9448
:102640004811101614F09FEF01C091E0989F902D53
:10265000112490933902112361F00E944811111640
:1026600014F09FEF01C091E0989F902D112490935A
:102670003A02309139023323E1F020913A022223C9
:10268000C1F045EB3403C0011124992319F0909354
:10269000390203C081E08093390235EB2303C00186
:1026A0001124992319F090933A0203C081E080939A
:1026B0003A028091370281110BC08091380281115A
:1026C00007C080913902811103C080913A028111C3
:1026D0000E945312EB82FC820D831E8386E0FE0172
:1026E0003196A5E3B2E001900D928A95E1F7269626
:1026F0000FB6F894DEBF0FBECDBFDF91CF911F9113
:102700000F91FF90EF900895E5E3F2E086E0DF019E
:102710001D928A95E9F710923302109232021092BC
:1027200034020895CF93DF93EC01FB01828188236B
:1027300009F43CC1C430FDE5DF0760F4CB3F9CE504
:10274000D90788F49E0122503C452431310508F018
:102750002EC109C0C236EDE5DE0729F0C63AFDE517
:10276000DF0709F024C10E94F10B9093550280937A
:102770005402C1318CE5D80709F4C6C008F042C044
:10278000C930ECE5DE0709F49BC000F5C5308CE5E7
:10279000D80709F485C078F4C330ECE5DE0709F406
:1027A00078C008F07AC0C230DC4509F0F5C08091ED
:1027B00054028160EFC0C7309CE5D90709F478C0A6
:1027C00008F07AC0809154028061E4C0CD30FCE50D
:1027D000DF0709F487C058F4CB309CE5D90709F42A
:1027E00079C008F07BC08091540288606FC0CF3000
:1027F000FCE5DF0709F480C008F082C08091540234
:10280000877FC8C0CE3F9CE5D90709F471C000F5A9
:10281000C531FCE5DF0709F485C068F4C3319CE5E8
:10282000D90709F475C008F095C00E94440680914C
:1028300054028F77AFC0CC3FFCE5DF07A9F108F069
:1028400054C0CB3FDC4509F0A7C08091550240C081
:10285000C230EDE5DE0709F489C058F4C1158DE5F5
:10286000D80709F45AC008F069C080915502826007
:102870002FC0C236EDE5DE0709F47CC0C63AFDE59F
:10288000DF0709F481C0C330DD4509F085C080E071
:102890006EC08091540282607DC08091540216C047
:1028A00080915402886076C08091550282604FC04A
:1028B0008091540280626EC08091540280646AC02C
:1028C0000E94440680915402806864C0846062C0A3
:1028D00081603DC0809154028E7F5CC08091540223
:1028E0008D7F58C08091540216C08091550218C047
:1028F000809155028D7F2BC0809154028F7E4AC0FB
:10290000809154028F7D46C0809154028F7B42C0DB
:1029100080915402877F8B7F3DC0809155028D7FCF
:102920008E7F15C08091540282FB222720F991E00E
:10293000922790FB82F990FB83F92CC0809155027D
:10294000982F909591708E7F892B90FB81F98093C1
:10295000550222C00E9444068091540287FB222720
:1029600020F991E0922790FB87F914C081E00E9442
:10297000880C12C08091540284FB222720F991E038
:10298000922790FB84F906C080915402982F90956D
:1029900090FB80F9809354028091540290915502EB
:1029A0000E94020C0E94440680E001C081E0DF9199
:1029B000CF910895CF93DF9386319C4541F5EB018C
:1029C0000E94B50B982F8A8120910201309103015A
:1029D000882379F09A7A81E009F480E080933B02C1
:1029E000911102C069E201C065E3C9010E9461164C
:1029F0000AC080913B02811102C069E201C065E317
:102A0000C9010E9463160E94860B80E001C081E02C
:102A1000DF91CF9108950F931F93CF93DF93C42F2E
:102A2000D22FFC0182818823C9F040933E020E948C
:102A3000081790933D0280933C0280E28C0F88300F
:102A400008F057C0C77081E001C0880FCA95EAF747
:102A5000DF91CF911F910F910C94220480913E023F
:102A6000481330C080913C0290913D020E94201793
:102A7000883C910538F510E21D0FCD17B9F080E2C2
:102A80008C0F883040F4C77081E001C0880FCA9570
:102A9000EAF70E942904183028F581E09D2F9770ED
:102AA00001C0880F9A95EAF70E942204802F0E94A5
:102AB00019041830F0F4D77081E001C0880FDA955E
:102AC000EAF70AC080E28C0F883098F4C77081E082
:102AD00001C0880FCA95EAF7DF91CF911F910F913E
:102AE0000C942904802FDF91CF911F910F910C94AA
:102AF0001904DF91CF911F910F9108950F939C01BD
:102B0000CB01243F4CE5340731F188F4293DFCE545
:102B10003F07D9F02A3D4CE5340779F1283D3C4583
:102B2000A9F506E221EE41EE68ED7CE52BC0263FDB
:102B3000FCE53F07E1F0A8F0273F3C4539F507E207
:102B400025EE46EE67EF7CE51DC007E225EE45EE7B
:102B500069ED7CE517C006E221EE40EE64EF7CE50E
:102B600011C007E225EE44EE65EF7CE50BC006E2FE
:102B700021EE42EE66EF7CE505C008E221E045EE7D
:102B80006AED7CE50E940B1580E008C0FC018281A3
:102B9000882319F010923E0201C081E00F91089540
:102BA00090939101809390010895909344028093B3
:102BB00043020895E0914302F0914402309721F0DE
:102BC0000190F081E02D099480E00895E0914302A6
:102BD000F0914402309721F00280F381E02D0994B6
:102BE0000895E0914302F0914402309739F022E0D9
:102BF000DC012C930480F581E02D09940895209147
:102C00004102309142022817390771F09093420235
:102C100080934102E0914302F0914402309721F009
:102C20000680F781E02D0994089520913F023091AC
:102C300040022817390771F09093400280933F02B9
:102C4000E0914302F0914402309721F00084F18535
:102C5000E02D09940895662349F0FC013296089608
:102C60002191621729F0E817F907D1F780E008955C
:102C700081E008959C01FC0132969FEF80E0419134
:102C8000461789F09F3F19F4411101C0982F8F5FBB
:102C90008630A9F79F3F39F0F901E90FF11D97FD43
:102CA000FA956283089508959C012A5F3F4FFC01C5
:102CB0004281461301C01282019682179307B9F729
:102CC00008950C943A160C945416029626E0FC01D2
:102CD00011922A95E9F7089508950C946C1683E0F3
:102CE000809345020C946D16811102C081E001C0F1
:102CF00082E0809345020C946D160C94741681E06A
:102D0000809345020C946D160C947F1608950C94D4
:102D100086160C9487160C9486160C9486160C94C2
:102D20008616CF930E948D160E946A100E948B1601
:102D3000C0E08C2F0E94940F892B29F4CF5FC530FF
:102D4000C1F780E001C081E0CF91089508951F92FE
:102D50000F920FB60F9211248F939F93AF93BF934F
:102D600080914602811113C080916A0290916B029A
:102D7000A0916C02B0916D024196A11DB11D80938E
:102D80006A0290936B02A0936C02B0936D02BF91A4
:102D9000AF919F918F910F900FBE0F901F9018953C
:102DA00080917202843031F10E94750210924602C5
:102DB00020E488E190E00FB6F894A8958093600035
:102DC0000FBE2093600083B7817F846083BF83B789
:102DD000816083BF7894889583B78E7F83BF0FB659
:102DE000F894A895809160008861809360001092AB
:102DF00060000FBE08950E9444060C94790282E0A0
:102E000084BD93E095BD9AEF97BD80936E000895C1
:102E10002FB7F89480916A0290916B02A0916C0296
:102E2000B0916D022FBF08952FB7F89460916A0298
:102E300070916B0280916C0290916D022FBF08958A
:102E40009C014FB7F89480916A0290916B02A09117
:102E50006C02B0916D024FBF821B930B0895789462
:102E60001F920F920FB60F9211248F939F93AF93DF
:102E7000BF9380916A0290916B02A0916C02B09115
:102E80006D020196A11DB11D80936A0290936B02A1
:102E9000A0936C02B0936D02BF91AF919F918F91FF
:102EA0000F900FBE0F901F90189581E08093E00067
:102EB00080E28093D8001092C9008FE19EE40197D0
:102EC000F1F700C0000087E090EBDC0180937B020B
:102ED00090937C02A0937D02B0937E029CE088E1F7
:102EE0000FB6F894A895809360000FBE9093600091
:102EF000FFCF809152020895089522E02093E900C7
:102F00002FEF3091E800215035FD06C035ED3A95A0
:102F1000F1F700002111F5CF2091E80025FF0BC04B
:102F200040E050E066E070E00E94A7198091E80060
:102F30008E778093E8000895CF93DF9321E020936C
:102F4000E9002FEF3091E800215035FD06C035ED46
:102F50003A95F1F700002111F5CF2091E80025FF07
:102F600014C0EC0140E050E068E070E00E94A71956
:102F70008091E8008E778093E80088E0FE01AAE463
:102F8000B2E001900D928A95E1F7DF91CF9108951B
:102F900080934702709349026093480280917202C5
:102FA000843001F582E08093E9008FEF9091E80092
:102FB000815095FD06C095ED9A95F1F700008111BD
:102FC000F5CF8091E80085FF0DC040E050E063E060
:102FD00070E087E492E00E94A7198091E8008E7764
:102FE0008093E8000895BC0184E00C94C817BC01EC
:102FF00083E00C94C81780917102811109C00E946E
:10300000381B0E94951B8091E20084608093E2004F
:1030100008951092710208950C94841660916E02C6
:1030200081E0611101C080E00C946F1690917202F2
:1030300081E0943009F080E060916E020C94741687
:1030400042E061EC81E00E94B11A42E261EC82E070
:103050000E94B11A9091720281E0943009F080E0F0
:1030600060916E020C947D1680917402833009F495
:1030700061C030F4813071F0823009F49AC0089553
:103080008A3009F486C08B3009F46CC0893009F0AD
:10309000A8C020C080917302813A09F0A2C080913B
:1030A000E800877F8093E800809177029091780212
:1030B000892B21F468E08AE492E003C060E080E0BC
:1030C00090E070E00E94F2198091E8008B77809385
:1030D000E800089580917302813209F082C08091E6
:1030E000770290917802029708F07BC08091E80007
:1030F000877F8093E8008091E80082FD05C0809181
:1031000072028111F8CF6DC02091F3008091F2001E
:1031100090E0922B029731F48091F100813011F010
:10312000863021F48091F100809352028091E80072
:103130008B7753C080917302813A09F052C080911D
:10314000770290917802892B09F04BC08091E800BA
:10315000877F8093E8008091E80080FFFCCF80911A
:10316000180136C0809173028132D9F580917702BF
:1031700090917802892BA9F58091E800877F809350
:10318000E8000E94E61A80917502809318010C9461
:10319000440680917302813221F58091E800877F97
:1031A0008093E8000E94E61A809176028093530291
:1031B000089580917302813AA1F48091E800877F9D
:1031C0008093E8008091E80080FFFCCF809153025B
:1031D0008093F1008091E8008E778093E8000C9452
:1031E000E61A089584B7877F84BF0FB6F894A89530
:1031F00080916000886180936000109260000FBE33
:1032000090E080E80FB6F89480936100909361009D
:103210000FBE0C947F160E94381B0E94951BE2EE95
:10322000F0E080818460808378940C942A1E8CE086
:1032300091E00C94D515809172028530A9F48091AB
:103240007202853079F40E94D01680917002882332
:10325000B1F30E949116882391F30E9491190E9464
:103260004406EDCF0C94FB16089508950C9438197C
:10327000292F332723303105C9F060F4213031057F
:1032800081F02230310509F044C08BE390E028E260
:1032900032E043C021323105E1F02232310549F1FB
:1032A00038C082E190E023E632E037C099278130D0
:1032B000910549F028F0029761F5E4E0F2E005C0DD
:1032C000E4E2F2E002C0E2E1F2E0849190E09F01EA
:1032D00024C06115710541F061307105D1F489E0B8
:1032E00090E023E532E019C089E090E02AE332E083
:1032F00014C06115710541F06130710551F48BE71F
:1033000090E025E732E009C080E490E020EF32E071
:1033100004C080E090E020E030E0FA0131832083B7
:10332000089580E189BD82E189BD09B400FEFDCF29
:103330008091D8008F7D8093D8008091E0008260DA
:103340008093E0008091E00081FDFCCF0895CF9252
:10335000DF92EF92FF920F931F93CF93DF93EC01D5
:103360008B017A010E94051B811133C0E114F10425
:1033700039F0F70180819181081B190BC80FD91F03
:10338000C12CD12C0115110519F18091E80085FDA2
:1033900016C08091E8008E778093E800E114F10474
:1033A00049F0F70180819181C80ED91ED182C08277
:1033B00085E00FC00E94051B882321F30AC0899174
:1033C0008093F10001501109FFEFCF1ADF0ADACF25
:1033D00080E0DF91CF911F910F91FF90EF90DF90F0
:1033E000CF9008952091790230917A0226173707FD
:1033F00048F06115710539F42091E8002E7720938B
:10340000E80001C0B901FC0120E06115710579F106
:10341000809172028823F1F18530F1F18091E8000A
:1034200083FD3CC08091E80082FD2EC08091E800C1
:1034300080FFEBCF2091F3008091F20090E0922B7F
:103440006115710551F08830910538F42191209370
:10345000F100615071090196F3CF21E0089709F05E
:1034600020E08091E8008E778093E800CECF211194
:10347000CFCF0AC080917202882361F0853061F05D
:103480008091E80083FD0AC08091E80082FFF2CFBE
:1034900080E0089582E0089583E0089581E0089532
:1034A0002091790230917A022617370748F061158A
:1034B000710539F42091E8002E772093E80001C0CF
:1034C000B901FC0120E06115710591F18091720252
:1034D000882309F440C0853009F43FC08091E8009A
:1034E00083FD3DC08091E80082FD2FC08091E800FF
:1034F00080FFE9CF2091F3008091F20090E0922BC1
:103500006115710559F08830910540F4249120939C
:10351000F1003196615071090196F2CF21E00897D0
:1035200009F020E08091E8008E778093E800CBCF0F
:103530002111CCCF0AC080917202882361F08530BE
:1035400061F08091E80083FD0AC08091E80082FF6D
:10355000F2CF80E0089582E0089583E0089581E04D
:103560000895982F973068F59093E900981739F0EF
:103570007091EC002091ED005091F00003C0242FD9
:10358000762F50E021FD02C09F5FECCF3091EB0021
:103590003E7F3093EB003091ED003D7F3093ED00A6
:1035A0003091EB0031603093EB007093EC0020938E
:1035B000ED005093F0002091EE0027FDE5CF80E074
:1035C00008958F708093E90081E0089580917302DF
:1035D00087FF11C08091E80082FD05C080917202D2
:1035E0008111F8CF11C08091E8008B770BC08091DA
:1035F0007202882349F08091E80080FFF8CF809123
:10360000E8008E778093E80008952091E4003091DF
:10361000E50095E64091EC00842F817040FF23C0C7
:103620008091E80080FD1DC080917202882399F08E
:10363000853099F08091EB0085FD11C04091E40048
:103640005091E5002417350729F3915011F09A01A4
:10365000E1CF84E0089582E0089583E0089581E059
:10366000089580E008954091E80042FFDDCF08957D
:103670000E94A61B0E94AE1BE0EEF0E080818160FC
:103680008083E8EDF0E080818F77808319BCA7ED1F
:10369000B0E08C918E7F8C9380818F7E808310929E
:1036A000710208950F931F93CF93DF930E94A61B7F
:1036B0000E94AE1BC8EDD0E088818F778883888117
:1036C0008068888388818F7D888319BC10927202FC
:1036D00010926E021092700210926F0200EE10E0D3
:1036E000F80180818B7F808388818160888342E0BC
:1036F00060E080E00E94B11AE1EEF0E080818E7F10
:103700008083E2EEF0E08081816080838081886048
:103710008083F80180818E7F8083888180618883A7
:10372000DF91CF911F910F910895E8EDF0E0808136
:103730008F7E8083E7EDF0E080818160808384E08C
:1037400082BF81E0809371020C94521BE8EDF0E09F
:1037500080818E7F80831092E20008951092DA00BB
:103760001092E10008951F920F920FB60F9211244C
:103770002F933F934F935F936F937F938F939F9379
:10378000AF93BF93EF93FF938091E10082FF0BC053
:103790008091E20082FF07C08091E1008B7F8093DF
:1037A000E1000E94291E8091DA0080FF1FC08091F5
:1037B000D80080FF1BC08091DA008E7F8093DA00F2
:1037C0008091D90080FF0DC080E189BD82E189BD73
:1037D00009B400FEFDCF81E0809372020E94FB17C6
:1037E00005C019BC109272020E9409188091E10074
:1037F00080FF19C08091E20080FF15C08091E20037
:103800008E7F8093E2008091E20080618093E200ED
:103810008091D80080628093D80019BC85E08093A5
:1038200072020E940E188091E10084FF30C08091E6
:10383000E20084FF2CC080E189BD82E189BD09B42A
:1038400000FEFDCF8091D8008F7D8093D8008091BD
:10385000E1008F7E8093E1008091E2008F7E809373
:10386000E2008091E20081608093E20080916E022C
:10387000882311F084E007C08091E30087FD02C037
:1038800081E001C083E0809372020E94161880914B
:10389000E10083FF29C08091E20083FF25C0809171
:1038A000E100877F8093E10082E0809372021092B2
:1038B0006E028091E1008E7F8093E1008091E200B2
:1038C0008E7F8093E2008091E20080618093E2002D
:1038D00042E060E080E00E94B11A8091F0008860D0
:1038E0008093F0000E940C18FF91EF91BF91AF916F
:1038F0009F918F917F916F915F914F913F912F9108
:103900000F900FBE0F901F9018951F920F920FB639
:103910000F9211242F933F934F935F936F937F9355
:103920008F939F93AF93BF93CF93DF93EF93FF93C7
:10393000C091E900CF708091EC00D82FD17080FD4C
:10394000D0E81092E9008091F000877F8093F0002A
:1039500078940E94C91C1092E9008091F000886060
:103960008093F000CD2BCF70C093E900FF91EF91D1
:10397000DF91CF91BF91AF919F918F917F916F9187
:103980005F914F913F912F910F900FBE0F901F901D
:1039900018951F93CF93DF93CDB7DEB7AA970FB6D5
:1039A000F894DEBF0FBECDBFE3E7F2E08091F100F7
:1039B000819322E0EB37F207C9F70E943418809117
:1039C000E80083FF2EC18091730290917402492F09
:1039D00050E04A30510508F024C1FA01EE59FF4F7A
:1039E0000C94591E803821F0823809F01AC108C0A1
:1039F00080916F0290917002992389F082600FC0CC
:103A0000809177028F70873008F00BC18093E900B6
:103A10008091EB0085FB882780F91092E900909156
:103A2000E800977F9093E8008093F1001092F100F6
:103A3000D1C0282F2D7F09F0F4C0882319F08230DF
:103A400061F0EFC080917502813009F0EAC09330D7
:103A500009F080E0809370022EC080917502811180
:103A60002AC0809177028F702FEF280F263008F040
:103A7000D8C08093E9002091EB0020FF1CC0933058
:103A800021F48091EB00806214C09091EB00906172
:103A90009093EB0021E030E0A90102C0440F551FD4
:103AA0008A95E2F74093EA001092EA008091EB00D9
:103AB00088608093EB001092E9008091E800877F96
:103AC0008093E8000E94E61AACC08111AAC0109150
:103AD00075021F778091E3008078812B8093E3004B
:103AE0008091E800877F8093E8000E94E61A809129
:103AF000E80080FFFCCF8091E30080688093E300C2
:103B0000111102C082E001C083E08093720289C07B
:103B10008058823008F085C08091750290917602BD
:103B20008C3D53E0950779F583E08A838AE28983A7
:103B30004FB7F894DE01139620E03EE051E2E32F08
:103B4000F0E050935700E49120FF03C0E295EF703E
:103B50003F5FEF708E2F90E0EA3010F0C79601C003
:103B6000C0968D939D932F5F243149F74FBF80916D
:103B7000E800877F8093E8006AE270E0CE0101965A
:103B80000E94F21916C06091770270917802AE011E
:103B90004F5F5F4F0E943619BC01892B09F441C069
:103BA0009091E800977F9093E80089819A810E9424
:103BB000501A8091E8008B778093E80032C08038FB
:103BC00081F58091E800877F8093E80080916E0204
:103BD0008093F1008091E8008E7772CF811121C02F
:103BE000809175029091760299270297D4F4809182
:103BF000E800877F8093E8008091750280936E02D1
:103C00000E94E61A80916E02811106C08091E30045
:103C100087FD02C081E001C084E0809372020E94AF
:103C200020188091E80083FF0AC08091E800877F18
:103C30008093E8008091EB0080628093EB00AA966D
:103C40000FB6F894DEBF0FBECDBFDF91CF911F91AD
:103C500008950895CF93809172028823A1F0C091B6
:103C6000E900CF709091EC00892F817090FD80E881
:103C7000C82B1092E9008091E80083FD0E94C91CC6
:103C8000CF70C093E900CF91089597FB072E16F4EB
:103C9000009407D077FD09D00E945F1E07FC05D075
:103CA0003EF4909581959F4F0895709561957F4F53
:103CB0000895EE0FFF1F0590F491E02D0994AA1BC3
:103CC000BB1B51E107C0AA1FBB1FA617B70710F007
:103CD000A61BB70B881F991F5A95A9F78095909539
:103CE000BC01CD010895FB01DC0104C08D91019060
:103CF000801921F441505040C8F7881B990B089552
:103D0000F999FECF92BD81BDF89A992780B50895A3
:103D1000A8E1B0E042E050E00C94B41E262FF999DF
:103D2000FECF92BD81BDF89A019700B4021639F01A
:103D30001FBA20BD0FB6F894FA9AF99A0FBE0895EB
:103D40000396272F0E948F1E0E948E1E252F0E94F1
:103D50008F1E242F0C948F1E0196272F0E948F1EDA
:103D60000C948E1EDC01CB01FC01F999FECF06C03C
:103D7000F2BDE1BDF89A319600B40D924150504029
:083D8000B8F70895F894FFCF95
:103D8800C8000E02280850011E0A140179179C1752
:103D98007D17F717F3177C1701E200E900EA00B571
:103DA80000B600B700CD008301CC008A01920194CF
:103DB800012102230224022502260227022A02B335
:103DC80000B4006F007000818283E200E900EA001D
:103DD800B500B600B700CD008301CC008A0192017E
:103DE80094012102230224022502260227022A0224
:103DF800B300B4006F007000818283909192939514
:103E08009496973435366667C6F1373332313000C9
:00000001FF
